:100000000C9493010C94CB010C94CB010C94CB0178
:100010000C94CB010C94CB010C94CB010C94CB0130
:100020000C94CB010C94CB010C94ED190C94BF1AD9
:100030000C94FF140C94CB010C94CB010C94CB01C9
:100040000C94CB010C94CB010C94CB010C94CB0100
:100050000C94CB010C9487150C94CB010C94CB0120
:100060000C94CB010C94CB010C94CB010C94CB01E0
:100070000C94CB010C94CB010C94CB010C94CB01D0
:100080000C94CB010C94CB010C94CB010C94CB01C0
:100090000C94CB010C94CB010C94CB010C94CB01B0
:1000A0000C94CB010C94CB010C94CB01E303E30340
:1000B0000F040F047704A205A205A20595042E05DE
:1000C0003F053F052C1B531B4B1C531B4B1C9F1BFD
:1000D000C21B4B1C191C281C29001E001F002000DD
:1000E00021002200230024002500260027002D00E7
:1000F0002E002A00000049004A002B0014001A00BC
:100100000800150017001C0018000C001200130056
:100110002F00300031004C004D0000003900040079
:100120001600070009000A000B000D000E000F006A
:100130003300340000002800000000000000E1004F
:1001400000001D001B000600190005001100100032
:10015000360037003800E5000000520000000000C3
:10016000E000E300E2000000000000002C000000BE
:1001700000000000E6000151E400500051004F0073
:10018000000001003A003B003C003D003E003F0003
:1001900040004100420043004400450001000000CF
:1001A0000100010001000100010001000100010047
:1001B0000100010001000100010001000100010037
:1001C0000100010000000100010001000100010028
:1001D0000100010001000100010001000100000018
:1001E000010000000000000001000000010001000B
:1001F00001000100010001000100010001000100F7
:1002000001000000010000000000010001000100E9
:1002100000000000000001000000000000000100DC
:100220000100010001000100010000001C03530057
:1002300061006B00610036003800200053006F0041
:100240006C006400650072000000160343004D005E
:100250004D002E00530074007500640069006F00AB
:1002600000000403090409023B00020100A0FA098E
:1002700004000001030101000921110100012240D5
:1002800000070581030800010904010001030000C3
:10029000000921110100012232000705820320001C
:1002A0000112010002000000084D434B5301000100
:1002B00002000105010980A101850319012AB70087
:1002C000150126B700950175108100C0050C0901C4
:1002D000A101850419012AA002150126A002950199
:1002E00075108100C005010906A101050719E02963
:1002F000E7150025019508750181029501750881B2
:10030000010507190029FF150026FF00950675084D
:1003100081000508190129059505750191029501CE
:1003200075039101C00011241FBECFEFDAE0DEBFDC
:10033000CDBF04B603FE18C080918D0290918E024D
:10034000A0918F02B09190028730904BA740B04BA4
:1003500059F410928D0210928E0210928F02109218
:100360009002E0E0F8E3099511E0A0E0B1E0ECEAEA
:10037000F9E302C005900D92AA38B107D9F722E03F
:10038000AAE8B1E001C01D92AD38B207E1F70E94C2
:10039000DD110C94D41C0C94000081E0089581E0E0
:1003A00008950C94CF0108950C94D3011F93CF931B
:1003B000DF9300D000D01F92CDB7DEB749835A83B8
:1003C0006B8330918D0189819A81311114C066232C
:1003D00059F0222349F00E94DB07182F682F8981EA
:1003E0009A810E94840703C00E94AF07182F698179
:1003F0007A81812F04C00E94DB0769817A810F9086
:100400000F900F900F900F90DF91CF911F910C9450
:10041000270FFC01262F40815181628173818481E5
:100420000C94D60181E00895CF93DF93EC0160E056
:100430000E940902BE01DF91CF910C94D4010C946B
:1004400070100C946C1008950E942E060E942302D6
:100450002FEF84E39CE0215080409040E1F700C002
:1004600000000C94AD150F931F93CF93DF938C0175
:1004700061E00E940902EC01B8010E94D1018823C9
:10048000F1F1B801CE010E94D6138823C1F1B80161
:10049000CE010E94EA11882391F1B801CE010E9499
:1004A0003213882361F1F8018281882309F1CB3569
:1004B0008DE5D807C1F050F4C115FCE5DF0781F0E8
:1004C000CF3DDC45A9F40E94120D19C0CC35EDE5F5
:1004D000DE0761F0CD35DD4559F40E94550C08C0AA
:1004E0000E9424020CC00E945E0C02C00E94610C9B
:1004F000C801DF91CF911F910F910C94CD0180E045
:10050000DF91CF911F910F9108950E94DF140C94F9
:100510009E020E94A1020C94E51408950C948D0291
:1005200081E008950C9490020895CF93C82F0E9403
:100530008E028C2F0E949202CF91089580E00C943D
:1005400095020E9432140C9495020E9432149091EC
:100550008C01891721F080938C010C9495020895E9
:10056000CF93DF93CDB7DEB72B970FB6F894DEBFEE
:100570000FBECDBF4F83588769877A878B876111FC
:100580000E94A10B9E012F5F3F4F86E0F90111925F
:100590008A95E9F785E0FE013796D90101900D9221
:1005A0008A95E1F789819A814C815D81452B31F0F3
:1005B0009F3F31F491E08F3F19F403C091E001C0F7
:1005C00090E090FF09C049815A816B817C818D81C7
:1005D0009E810E94C20A05C0C9010E9412028111B7
:1005E000F2CF2B960FB6F894DEBF0FBECDBFDF91D2
:1005F000CF910895FC01808191810E941D0808958A
:10060000CF93882309F448C0C82F8CEF8C0F813A10
:10061000D0F46C2F80910201909103010E9481140B
:10062000882349F06C2F80910201909103010E9470
:10063000B9140E94C30B6C2F8091020190910301A9
:100640000E94B7140CC080E28C0F883058F4C77039
:1006500081E001C0880FCA95EAF70E94840BCF9110
:100660000C94C30BEBE5EC0FE33040F4F0E0E15CFD
:10067000FE4F808190E0CF910C944914C85AC73145
:1006800058F4EC2FF0E0EE0FFF1FEF5EFE4F80817D
:100690009181CF910C945F14CF910895882349F1F3
:1006A000682F8CEF860F813A38F480910201909187
:1006B00003010E94B9140CC080E2860F883050F408
:1006C000677081E001C0880F6A95EAF70E948A0B83
:1006D0000C94C30B8BE5860F833020F480E090E010
:1006E0000C944914685A673120F480E090E00C942F
:1006F0005F1408951F93CF93DF93182FEB010E948F
:100700000003209741F08FE99FE00197F1F700C0C7
:1007100000002197F6CF812FDF91CF911F910C948C
:100720004E03893319F060E070E002C060E570E0CC
:100730000C947A03882321F00E94840B0C94C30B41
:100740000895882321F00E948A0B0C94C30B08950E
:10075000CF92DF92EF92FF920F931F93CF93DF938D
:100760007C01D62FC72FFC011281058102950F70E5
:100770000E947A0B8823B9F01123A9F08C2F807F77
:10078000803421F080E28D0F883068F08091530230
:1007900082FD09C082E00E94230C0E947A0B91E046
:1007A000D82ED92601C0D12CCC2EC2948FE0C822DD
:1007B0008C2D90E08C30910508F0C4C1FC01EA5A00
:1007C000FF4F0C947F1C8C2F807FCF70882311F0FB
:1007D000C295C07F112399F0CC2309F49FC180E218
:1007E0008D0F883010F0D11104C08C2F0E94840B23
:1007F00003C08C2F0E94940B0E94C30B8FC18D2FBE
:100800000E944E03CC2309F49DC180E28D0F8830F5
:1008100038F1DD2329F18C2F0E949A0B24C08C2FF4
:10082000807FCF70803211F0C295C07FDD2319F038
:10083000D130A1F13DC08091530282FF17C0112336
:1008400049F0CC2329F08C2F0E94840B0E94C30B0B
:1008500080E065C180E00E944E03CC2309F472C1A0
:100860008C2F0E948A0B0E94C30B6CC1112371F064
:10087000002341F0013031F40E94A40B8C2B0E9424
:10088000AC0B60C10E94A40B8C2B1DC0002319F07F
:10089000013009F457C10E94B90B25C0112321F082
:1008A000063008F04FC10EC0053008F04BC11BC028
:1008B000112361F0002331F0F701858180FF2EC103
:1008C0008F7085838C2F0E949A033CC1002359F0BE
:1008D000D93309F034C1FFEF07EE13E0F1500040C7
:1008E0001040E1F72AC18C2F0E94A1032BC18C2F4D
:1008F00086958695837019F0813061F023C11123AC
:1009000021F08D2F9C2F937002C080E090E00E9418
:10091000491420C1112321F08D2F9C2F937002C008
:1009200080E090E00E945F1415C18C2F837009F065
:1009300047C011110BC12D2F229526952770220F2C
:10094000220F6D2F6F70862F90E0A0E0B0E0022E96
:1009500004C0880F991FAA1FBB1F0A94D2F7D4FFA7
:1009600010C04FE050E060E070E004C0440F551F3D
:10097000661F771F2A95D2F7409550956095709520
:1009800003C040E050E0BA01C695C695C3708A0125
:100990009B01082B192B2A2B3B2BC901B801C23014
:1009A00049F058F4C13019F00E949A06CFC00E9455
:1009B0008806CCC00E94AC06C9C00E948606C6C08C
:1009C000112319F08C2F817001C08695882309F4BA
:1009D000BDC02D2F229526952770220F220F6D2F37
:1009E0006F70862F90E0A0E0B0E0022E04C0880F68
:1009F000991FAA1FBB1F0A94D2F7D4FF10C04FE063
:100A000050E060E070E004C0440F551F661F771F80
:100A10002A95D2F7409550956095709503C040E0B7
:100A200050E0BA01C695C695C3708A019B01082B98
:100A3000192B2A2B3B2BC901B801C23049F058F4BD
:100A4000C13019F00E945F0781C00E944D077EC02F
:100A50000E9471077BC00E94C00678C0CF7011232E
:100A600039F08C2F0E94E6068D2F0E949A036EC0EB
:100A70008D2F0E94A1038C2F0E94070767C0D23FD1
:100A800021F128F4D03F41F0D13FC1F043C0D33F22
:100A900019F1D43F79F03EC0112341F0053008F040
:100AA00051C08C2F8F710E942C074CC0063008F06B
:100AB00049C0F7CF8091530282FF18C0112339F04B
:100AC0008C2F8F710E94E6063DC01123C9F38C2F35
:100AD0008F710E94070736C0112329F08C2F8F7168
:100AE0000E94D1062FC00E94CC062CC0112349F0D1
:100AF000CF718C2F0E94E60663E08C2F0E94080CB9
:100B000021C081E00E94230C0230E0F082E00E94CC
:100B1000230C18C0112331F0002391F28D2F0E9475
:100B2000000310C0002399F2D93349F41FEF27EED8
:100B300033E0115020403040E1F700C000008D2F1D
:100B40000E944E0388EF8C0D843020F40E943214F2
:100B50000E949502DD20C9F00E94760B80FD15C031
:100B6000F70112820E94700B0E94E606C7010E94E4
:100B7000E6050E94700BDF91CF911F910F91FF90BE
:100B8000EF90DF90CF900C940707DF91CF911F91EA
:100B90000F91FF90EF90DF90CF9008950F931F93E8
:100BA000CF93DF93EC01688179818A810E942808C4
:100BB0008C010E9483070E947406B801CE010E9436
:100BC000A803DF91CF911F910F910895CF93DF93E9
:100BD000EC01988189812B813C81232B31F08F3F5F
:100BE00031F481E09F3F19F403C081E001C080E04F
:100BF00080FD1DC0CE010E943302811110C00E94F1
:100C00007A0B8823A1F08A81882389F0809153028E
:100C100082FD0DC082E0DF91CF910C94230CCE01B8
:100C20000E94CE05CE01DF91CF910C941402DF918A
:100C3000CF91089580E090E00E94491480E090E018
:100C40000E945F140E94A10B0C94C30B80910201BF
:100C5000909103010E94BB140C941A060E94910B00
:100C60000C94260692959F70963079F010F492506D
:100C700001C09A50923068F4803F69F018F4883EC1
:100C800040F409C0843F29F406C0883E20F0813F2B
:100C900011F080E0089581E00895FC018081918148
:100CA0000E941D080E9432060895CF93DF9300D062
:100CB00000D01F92CDB7DEB70F900F900F900F901E
:100CC0000F90DF91CF910895CF93DF9300D000D0A4
:100CD00000D0CDB7DEB726960FB6F894DEBF0FBEB4
:100CE000CDBFDF91CF910895089508950C947506B6
:100CF0000C9476060E9478066093C9017093CA012D
:100D00008093CB019093CC010C941A060C947A0634
:100D10000F931F930091C9011091CA012091CB013B
:100D20003091CC01602B712B822B932B1F910F9153
:100D30000C947A060F931F930091C9011091CA0178
:100D40002091CB013091CC01602371238223932326
:100D50001F910F910C947A060F931F930091C90174
:100D60001091CA012091CB013091CC0160277127ED
:100D7000822793271F910F910C947A060C94750685
:100D80000E94BE066093C5017093C6018093C7019F
:100D90009093C8010C941A0660E070E0CB010C94AB
:100DA000C0060F931F9341E050E060E070E08A01BD
:100DB0009B0104C0000F111F221F331F8A95D2F719
:100DC000C901B8011F910F910C94C0060F931F9396
:100DD00041E050E060E070E004C0440F551F661F22
:100DE000771F8A95D2F78091C5019091C601A09195
:100DF000C701B091C8018A019B01082B192B2A2B2E
:100E00003B2BC901B8011F910F910C94C0060F93A1
:100E10001F9341E050E060E070E004C0440F551FB4
:100E2000661F771F8A95D2F740955095609570950B
:100E30008091C5019091C601A091C701B091C801F0
:100E40008A019B01082319232A233B23C901B801E6
:100E50001F910F910C94C0060F931F9341E050E037
:100E600060E070E004C0440F551F661F771F8A952D
:100E7000D2F78091C5019091C601A091C701B091B0
:100E8000C8018A019B01082719272A273B27C90186
:100E9000B8011F910F910C94C0060F931F930091FE
:100EA000C5011091C6012091C7013091C801602B86
:100EB000712B822B932B1F910F910C94C0060F93D3
:100EC0001F930091C5011091C6012091C701309177
:100ED000C80160237123822393231F910F910C94E7
:100EE000C0060F931F930091C5011091C601209178
:100EF000C7013091C80160277127822793271F916E
:100F00000F910C94C006089521E1929F800D112449
:100F1000E82FE695E695E695877051E001C0550FFC
:100F20008A95EAF785E0E89FF0011124E257FE4F29
:100F300020E030E070E04081CB01022E02C09695A7
:100F400087950A94E2F78170819584278523842709
:100F500081932F5F3F4F2530310569F7089521E1D7
:100F6000929F800D1124682F669566956695982F3F
:100F7000977085E0689FB001112440E050E080E068
:100F8000FB01E40FF51FE257FE4F208130E0092EF0
:100F900002C0369527950A94E2F721703327042E74
:100FA00001C0220F0A94EAF7822B4F5F5F4F453052
:100FB000510531F70895BF92CF92DF92EF92FF92E1
:100FC0000F931F93CF93DF938C01C090C501D090F6
:100FD000C601E090C701F090C8018091C9019091CD
:100FE000CA01A091CB01B091CC01C82AD92AEA2A22
:100FF000FB2ACFE1D0E0D701C6010C2E04C0B69584
:10100000A795979587950A94D2F780FD04C02197FC
:1010100090F7B12C07C0BC2EB8018C2F0E943A0F5C
:101020000197A9F38B2DDF91CF911F910F91FF9025
:10103000EF90DF90CF90BF900895CF93DF93EC01B6
:101040000E94DB07BE010E943A0FDF91CF91089505
:101050001F93CF93DF93EB0190918D01992321F0A2
:10106000CB010E941D0813C0882349F0CB010E94C8
:10107000DB07182F682FCE010E94840704C0CB0124
:101080000E94AF07182FBE01812F0E943A0FDF91F7
:10109000CF911F9108951F93CF93DF93C091CD01FE
:1010A00016E08091CE01C81799F0D0E01C9FF001A6
:1010B0001D9FF00D1124E153FE4F4081518162814B
:1010C0007381848195810E9464062196C770E9CF5F
:1010D000DF91CF911F9108954091FF01509100023F
:1010E00060910102709102028091030290910402CA
:1010F0000C946406EF92FF920F931F93CF93DF93AC
:101100008091040282958F7009F065C08091010280
:10111000882309F460C08091CD01F090CE01109138
:10112000FF0100910002609102027091030291E0C0
:101130001F3F09F090E0C0910001D0910101292FDB
:1011400096E0E92E8F1509F446C06115710521F06E
:101150000F3F21F030E003C031E001C0322F90E0BA
:1011600030FD36C0E89EF001E99EF00D1124DF014C
:10117000A153BE4F11963C911197301329C03C9159
:10118000311326C012963C911297311121C013964B
:101190004D915C911497461B570B4C175D07C0F49B
:1011A000809104028F70806180930402EC52FE4FA4
:1011B00080818F70806180838FEF91E00E94E605CF
:1011C000DF91CF911F910F91FF90EF900C944B08FE
:1011D00001968770B7CFDF91CF911F910F91FF904C
:1011E000EF9008959F92AF92BF92CF92DF92EF92CD
:1011F000FF920F931F93CF93DF93CDB7DEB7619725
:101200000FB6F894DEBF0FBECDBF8C0185E0F801AC
:10121000DE011D9601900D928A95E1F7D801129694
:10122000EC909091FF01E091000220910202309138
:1012300003022115310531F0EF3F31F481E09F3F8A
:1012400019F403C081E001C080E0B82FB1709B2E7B
:1012500080FD47C1D8014C9111965C91119713966E
:10126000AD90BC9014978FEFC82E81E0D82EF090EF
:101270000102B501621B730B209100013091010145
:10128000FF2009F4D9C0809104026217730708F0A7
:1012900095C0282F207F09F052C05E1313C0491358
:1012A00011C0FE2CE1100EC08F708061809304028B
:1012B0000E946C08C6010E94E60580910402F801B4
:1012C00085834DC1AB2831F05F3F31F481E04F3F62
:1012D00019F403C081E001C080E080FD03C081E01B
:1012E0008E2502C080E090E0F82FF170FF2E80FF85
:1012F0001CC08091CD012091CE0136E0821709F407
:101300000BC190E0389FF001399FF00D1124E1539B
:10131000FE4F6181561306C06081461303C062818F
:10132000E61203C001968770E9CFFE2CEE2009F487
:1013300016C18091040281608093040254C05E1340
:1013400006C0491304C0E11002C0F80199C0C801E9
:101350000E944D06882361F1EE2051F12091040294
:10136000822F82958F7090E0029774F08091FF0138
:101370009091000298878F831986BB86AA862C8756
:10138000CE0107960E94E60586E0F801AFEFB1E0D6
:1013900001900D928A95E1F70E947A080E946C08EC
:1013A0000AC05E1711F1C8010E944D0681112CC0C0
:1013B000C8010E94E605FF24F394D1C0282F207FA6
:1013C00081F77A2DB98AA88A6E2D89890E945506DF
:1013D0008FEF91E00E94E60586E0D6011D928A9586
:1013E000E9F70E946C08F12CBAC04913DCCFE11078
:1013F000DACFF8018583C8010E94E60586E0D601B0
:101400001D928A95E9F7ABC0EE2091F2209104027B
:10141000822F82958F7090E002970CF4B5CF809167
:10142000FF01909100029A8389831B82BD82AC8266
:101430002E83CE010196A6CF6217730708F044C031
:10144000FE2CEE2009F4B4CF5E1330C049132EC039
:101450002091040220FD21C0822F82958F70482F99
:1014600050E041155105C9F0F80125834F30510571
:1014700041F08F5F982F9295907F822F8F70892BEC
:101480008583C8010E94E60586E0F801AFEFB1E070
:1014900001900D928A95E1F73CC086E0F801AFEF2C
:1014A000B1E001900D928A95E1F759C0C8010E9400
:1014B0004D06811169CF80910402816080930402FE
:1014C000C8010E94E6054BC07A2DB98AA88A6E2D04
:1014D00089890E94550686E0D6011D928A95E9F712
:1014E00018C0EE2009F464CFC8010E944D06F82E02
:1014F000882309F45DCF86E0F801AFEFB1E00190F9
:101500000D928A95E1F78FEF91E00E94FA020E9416
:101510007A080E946C0823C04D875E878D859E8562
:101520000E941D08292F22952F70223028F49F70C9
:1015300039F0811105C00BC0243028F49F7049F4A4
:10154000805E883020F0C8010E94E6059F2CF92CAF
:1015500006C0D80115969C91907F91F7F8CF8F2DFA
:1015600061960FB6F894DEBF0FBECDBFDF91CF916D
:101570001F910F91FF90EF90DF90CF90BF90AF90B1
:101580009F9008951F93CF93DF93CDB7DEB72C972D
:101590000FB6F894DEBF0FBECDBF4F835887698763
:1015A0007A878B879C87CE0107960E94F208882352
:1015B000D1F09F8188852A853B85232B31F08F3F91
:1015C00031F481E09F3F19F403C081E001C080E065
:1015D00080FD47C04F81588569857A858B859C85BC
:1015E0000E9464063EC086E0FE013796DE01119639
:1015F00001900D928A95E1F7FF81E8856A857B85E8
:101600006115710531F0EF3F31F481E0FF3F19F4CE
:1016100003C081E001C080E080FD23C02091CE01A5
:1016200030E0C9010196877099274091CD0150E0C3
:1016300084179507F1F1F983EA837D836C8396E043
:10164000929FD001939FB00D1124A153BE4FFE0174
:10165000319601900D929A95E1F78093CE010E9408
:101660004B0816E08091CD019091CE01891771F160
:10167000189FC001112481539E4F0E94F2088823B5
:1016800029F1E091CD011E9FF0011124E153FE4F9D
:101690004081518162817381848195810E946406B9
:1016A0008091CD0190E00196877099278093CD01BC
:1016B000D9CF0E942E061092CE011092CD01EFEFED
:1016C000F1E086E0DF011D928A95E9F72C960FB6CE
:1016D000F894DEBF0FBECDBFDF91CF911F9108956B
:1016E00080910D02859585958595089580910D02CF
:1016F0008770089590910D02977081E009F480E061
:10170000089580911802089590911802892B809372
:1017100018020895809590911802892380931802E9
:10172000089510921802089590911702892B8093C2
:1017300017020895809590911702892380931702CC
:10174000089510921702089580910E020895089549
:101750000C94A70B0C94A80B9091530292FD08C017
:1017600090910E02981721F080930E020C94AA0B10
:10177000089580910E02882329F010920E0280E0D5
:101780000C94AA0B0895CF93DF93E0910201F0919E
:101790000301809118028083E0910201F09103011E
:1017A000908180911702892B808380910E0288237B
:1017B00081F0E0910201F09103019081892B8083F7
:1017C00080910201909103010E94751481110E9481
:1017D000B90BC0910201D091030148E050E065E0EF
:1017E00072E0CE010E94851C892B69F088E0FE0121
:1017F000A5E0B2E001900D928A95E1F7CE01DF916C
:10180000CF910C943E14DF91CF9108950C94A70BC7
:101810009091530292FD10C098E0899F900111248D
:10182000262B20930D020E94E60680910D028595DD
:10183000859585950C94060C0C94E60610920D0285
:1018400080E00C94060C20910D02809582238093F9
:101850000D02982F977099F430E0482F082E000C55
:10186000550B2417350759F09091530292FD07C08C
:101870008595859585950E9407070C941E0C089503
:101880009091530292FB222720F9281769F080FBE0
:1018900092F99093530280915202909153020E94C8
:1018A0008E0C82E00C94230C08958091530282FBED
:1018B000882780F991E089270C94400C81E00C94F2
:1018C000400C80E00C94400C6FEF7FEF80E090E0E4
:1018D0000C94BE1C80E090E00E949A1C21E0893E9E
:1018E0009E4F09F020E0822F089582E090E00C9452
:1018F000921C83E090E00C94921CCF9384E090E0E3
:101900000E94921CC82F82E290E00E94921C2C2F11
:1019100030E0A901582BCA01CF910895CF93C92F68
:10192000682F84E090E00E94A01C6C2F82E290E07F
:10193000CF910C94A01CAB01BC018FE090E00C9403
:10194000B21CAB01BC0183E190E00C94B21C60E0DE
:1019500070E0CB010C94A10C60E070E0CB010E9420
:101960009B0C0C94A70C69EE7EEF80E090E00E9447
:10197000BE1C60E082E090E00E94A01C60E083E07A
:1019800090E00E94A01C1092C9011092CA0110920E
:10199000CB011092CC0160E084E090E00E94A01C9A
:1019A00060E082E290E00E94A01C60E085E090E0B0
:1019B0000E94A01C60E086E090E00E94A01C6FEFF7
:1019C00087E090E00E94A01C40E050E0BA0188E06F
:1019D00090E00E94B21C60E08DE090E00E94A01CAC
:1019E00040E050E0BA0188E190E00E94B21C60E063
:1019F00087E190E00E94A01C40E050E0BA018CE139
:101A000090E00E94B21C60E070E080E290E00E94F2
:101A1000BE1C40E050E0BA0188E190E00E94B21C98
:101A20000C94AC0C0C94B30C682F8EE090E00C94EA
:101A3000A01C0E946C156093310270933202809357
:101A400033029093340260932D0270932E028093A0
:101A50002F0290933002089585B7806885BF85B7BF
:101A6000806885BF089581E008950C94330D089532
:101A70000C94370D0C94370D0C943A0D0C94370DD3
:101A80000C943E0D0C94370D0E942C0D86E190E1D4
:101A90000E9428140E94420D0C94400D0E94380DA3
:101AA0000C94370D0E9430100C9494020E9457152C
:101AB0000E9434110E94520D0C943C0D2F923F92C3
:101AC0004F925F926F927F928F929F92AF92BF924E
:101AD000CF92DF92EF92FF920F931F93CF93DF93FA
:101AE000CDB7DEB72D970FB6F894DEBF0FBECDBFD2
:101AF0000E944911282E81110E94190D89E192E05E
:101B00009D878C8700E010E0302E802F0E945410BB
:101B10002B013C01EC85FD8581919191A191B191C1
:101B2000FD87EC875301420188269926AA26BB2609
:101B300081149104A104B104B1F40F5F1F4F05306B
:101B4000110511F78FEF89838A831B820E9460152C
:101B50008160782F9D838C8349815A816B818D812F
:101B60000E94B00251C08091350281FD0E94601038
:101B70001B86C12CD12C7601C394D501C4018C21C4
:101B80009D21AE21BF21892B8A2B8B2B91F10E94A5
:101B9000350D8823D1F0FB85FE833F824C205D20EC
:101BA0006E207F2081E045284628472809F480E000
:101BB00088870E9460158160782F9A8789874E8177
:101BC0005F8168858A850E94B002000F111F000F97
:101BD000111FF801E75EFD4F80819181A281B381E1
:101BE000C826D926EA26FB26C082D182E282F38269
:101BF0000BC08B858F5F8B87CC0CDD1CEE1CFF1C14
:101C0000813109F0BACF99CF81E0211001C080E085
:101C10002D960FB6F894DEBF0FBECDBFDF91CF91EA
:101C20001F910F91FF90EF90DF90CF90BF90AF90FA
:101C30009F908F907F906F905F904F903F902F90EC
:101C400008950E945E0D0C94A502CF93DF930E942D
:101C50003F0FEC01811522E59207E8F5811531E58A
:101C6000930708F0B6C0883E910528F5803E91059F
:101C700008F0E9C0883A910570F4853A910508F0BA
:101C80007AC08130910509F473C008F4D9C0049773
:101C900008F0D9C0D5C08F3B910508F0D1C0C85A13
:101CA000D0E0CC0FDD1FCE5BDE4F0990D881C02D78
:101CB000CE019464C9C0811540E5940708F069C05D
:101CC000811550E4950708F060C09A9581159F41F1
:101CD00008F4B9C0B5C0811536E5930728F581151C
:101CE00045E5940708F092C0811554E5950708F082
:101CF00087C0AC0143705527282F26952695C1151E
:101D0000D34508F06CC081E090E002C0880F991FB5
:101D10004A95E2F740E2249F90011124EC01C22B86
:101D2000D32BCE019C6890C081152AE5920780F4E0
:101D3000811539E5930708F072C0811548E59407CD
:101D400008F47EC0D82FCC27CE01806F906A7CC06B
:101D500090568115904208F073C08D2F8F710E94AC
:101D6000D30FDD27D0628F71AE01582BCA016CC032
:101D700081E090E069C0C55AD0E0C059DE4F88814B
:101D8000C82FD0E0CE0190645FC0DF70CE01906AB2
:101D90005BC074E0969587957A95E1F7282F2370BC
:101DA0003C2F337081E090E002C0880F991F3A9574
:101DB000E2F79C68AC01522B9A019C2F9F7096957C
:101DC000969550E2959FE0011124C9018C2B9D2B23
:101DD0003BC0D82FCC27CE01816F906A35C081E0FF
:101DE00090E002C0880F991F4A95E2F750E2259FC4
:101DF00090011124EC01C22BD32BCE019A6824C090
:101E0000D82FCC27CE01846F906A1EC00E94D30FBA
:101E10008F7190E0D82FCC27CE01906215C08F70C3
:101E20000E94D30F94E0D695C7959A95E1F7CF70AD
:101E3000D0E0DC2FCC27D0699E01282BC90104C03B
:101E400080E090E001C0CE01DF91CF91089525E5BB
:101E5000829FC0011124FC0121E1729FE00DF11D60
:101E60001124E60FF11DEE0FFF1FE852FF4F859181
:101E7000949108950E94270F0E94250E089582389C
:101E8000910569F1B0F48133910509F46DC048F40E
:101E90008932910509F463C08A32910509F469C059
:101EA00008958533910509F455C089339105B9F03A
:101EB0000895833E910569F138F4803E9105B1F0B3
:101EC000823E910509F10895863E9105A9F1873E6C
:101ED0009105B9F1843E910509F064C023C02091B9
:101EE000520220FD4FC021FD4DC008958091520245
:101EF00080FD44C08091530280FF44C08091520213
:101F000084FD42C083EE4DC08091520282FF38C0F2
:101F1000F5CF8091520282FD33C08091530280FD43
:101F200031C0ECCF8091530281FF32C080915202C8
:101F300084FD2AC087EE35C08091520283FF26C0FF
:101F4000F5CF8091520283FD21C08091530281FD23
:101F50001FC0ECCF8091520285FD1CC01DC0809136
:101F6000520285FD19C016C08091520286FD16C02E
:101F700017C08091520286FD13C010C089E311C0C2
:101F800082EE0FC080EE0DC080E00BC086EE09C06F
:101F900084EE07C089E205C085E303C08AE201C080
:101FA00081E390E008959091520292FF0DC0282F96
:101FB0002871283019F4877F846006C0282F247187
:101FC000243011F48B7F886093FF0DC0282F287177
:101FD000283119F4877E846106C0282F24712431AA
:101FE00011F48B7E88612091530220FF0DC0382FA1
:101FF0003871383019F4877F816006C0382F31710D
:10200000313011F48E7F886021FF0DC0282F287198
:10201000283119F4877E816106C0282F2171213172
:1020200011F48E7E886194FD877E089580E0089586
:102030000C94640C0E9449118FE39CE90197F1F71D
:1020400000C000000E94491180E00E94541060FF0F
:1020500004C00E9418100C94AD1508950C941A1029
:102060000E946A0C811102C00E94120D0E94750C20
:10207000809335020E947D0C90935302809352020C
:102080000E942E100E94790C682F70E080E090E092
:102090000E9486066091C5017091C6018091C701BA
:1020A0009091C8010C94BE0624E0829FC0011124C7
:1020B000FC01E859FD4F608171818281938108950F
:1020C000089580EA8A95F1F7089500C008950C9468
:1020D000611008950C9469100C946A100C946910A6
:1020E0000C946E10F894E82FE295EF70F0E031A1B7
:1020F000282F2F7081E090E001C0880F2A95EAF721
:10210000982F9095932391A392A1892B82A37894E1
:1021100008950F931F93CF93DF93C4E8D1E0899183
:102120008F3F11F00E94721081E0C938D807B9F7CB
:10213000C3E7D1E004E811E089918F3F11F00E94DC
:1021400072100C171D07C1F7DF91CF911F910F91EE
:1021500008954F925F926F927F928F929F92AF926B
:10216000BF92DF92EF92FF920F931F93CF93DF9373
:102170008C01C62FD0E0CE018C579E4F7C01FC0114
:1021800090819F3F09F460C0D62EF894E92FE29524
:10219000EF70F0E081A19F7021E030E001C0220FDC
:1021A0009A95EAF7822B81A382A12095282322A366
:1021B00078940E946510E3E7F1E024E831E0412CD7
:1021C000512C32014394812C912C540181918F3FE9
:1021D00099F0A82FA295AF70B0E090964C9150E086
:1021E0008F70BA0102C0759567958A95E2F760FD18
:1021F00003C0D301C20103C080E090E0DC01882A63
:10220000992AAA2ABB2A440C551C661C771C2E1737
:102210003F07E1F6F70180818F3F11F00E947210B5
:1022200061E081149104A104B10409F460E08D2DF2
:102230000E946710CC0FDD1FCC0FDD1FC00FD11F18
:1022400088829982AA82BB82DF91CF911F910F91E0
:10225000FF90EF90DF90BF90AF909F908F907F9016
:102260006F905F904F9008950E94891084E1E8E696
:10227000F2E0DF01982F1D929A95E9F7E4E5F2E08C
:10228000DF011D928A95E9F785E00E9494110C9474
:102290001F02FF920F931F93CF93DF93CDB7DEB74B
:1022A00064970FB6F894DEBF0FBECDBF8E010F5FEF
:1022B0001F4F84E1F80111928A95E9F7F12C6F2DF7
:1022C000C8010E94A910F394F5E0FF12F8CF44E191
:1022D00050E0B80184E592E00E94851CFF24F3944D
:1022E000009709F4F12C892B41F084E1F801A4E571
:1022F000B2E001900D928A95E1F72F2D45E068E656
:1023000072E084E592E00E9495110E9421028F2DD7
:1023100064960FB6F894DEBF0FBECDBFDF91CF91AC
:102320001F910F91FF9008950895FF920F931F93AF
:10233000CF93DF93F82ED92F8B01C42F222349F09E
:1023400081E0809338020E94601590933702809359
:102350003602809138028823F1F080913602909104
:1023600037020E9478150597B0F0EF2DFD2FD801A8
:1023700080E090E04C2F50E08417950754F40191D1
:102380001191219131910D931D932D933D930196C0
:10239000F3CF10923802DF91CF911F910F91FF90F0
:1023A00008950E9445170E94560D0C9451170E94E3
:1023B00055170E94210E0C946F170E94FE140E9464
:1023C0002C170E94440D0E94D1110E94D7110E9427
:1023D0004E0DFBCFCF93DF93EC01FB01828188236D
:1023E00009F43CC1C430FDE5DF0760F4CB3F9CE558
:1023F000D90788F49E0122503C452431310508F06C
:102400002EC109C0C236EDE5DE0729F0C63AFDE56A
:10241000DF0709F024C10E947D0C90935302809342
:102420005202C1318CE5D80709F4C6C008F042C099
:10243000C930ECE5DE0709F49BC000F5C5308CE53A
:10244000D80709F485C078F4C330ECE5DE0709F459
:1024500078C008F07AC0C230DC4509F0F5C0809140
:1024600052028160EFC0C7309CE5D90709F478C0FB
:1024700008F07AC0809152028061E4C0CD30FCE562
:10248000DF0709F487C058F4CB309CE5D90709F47D
:1024900079C008F07BC08091520288606FC0CF3055
:1024A000FCE5DF0709F480C008F082C08091520289
:1024B000877FC8C0CE3F9CE5D90709F471C000F5FD
:1024C000C531FCE5DF0709F485C068F4C3319CE53C
:1024D000D90709F475C008F095C00E942E068091B6
:1024E00052028F77AFC0CC3FFCE5DF07A9F108F0BF
:1024F00054C0CB3FDC4509F0A7C08091530240C0D7
:10250000C230EDE5DE0709F489C058F4C1158DE548
:10251000D80709F45AC008F069C08091530282605C
:102520002FC0C236EDE5DE0709F47CC0C63AFDE5F2
:10253000DF0709F481C0C330DD4509F085C080E0C4
:102540006EC08091520282607DC08091520216C09E
:1025500080915202886076C08091530282604FC0A1
:102560008091520280626EC08091520280646AC083
:102570000E942E0680915202806864C0846062C00E
:1025800081603DC0809152028E7F5CC0809152027A
:102590008D7F58C08091520216C08091530218C09E
:1025A000809153028D7F2BC0809152028F7E4AC052
:1025B000809152028F7D46C0809152028F7B42C033
:1025C00080915202877F8B7F3DC0809153028D7F27
:1025D0008E7F15C08091520282FB222720F991E064
:1025E000922790FB82F990FB83F92CC080915302D3
:1025F000982F909591708E7F892B90FB81F9809315
:10260000530222C00E942E068091520287FB22278D
:1026100020F991E0922790FB87F914C081E00E9495
:10262000140D12C08091520284FB222720F991E000
:10263000922790FB84F906C080915202982F9095C2
:1026400090FB80F980935202809152029091530244
:102650000E948E0C0E942E0680E001C081E0DF9176
:10266000CF910895CF93DF9386319C4541F5EB01DF
:102670000E94810B982F8A812091020130910301E1
:10268000882379F09A7A81E009F480E08093390216
:10269000911102C069E201C065E3C9010E94B7144B
:1026A0000AC080913902811102C069E201C065E36C
:1026B000C9010E94B9140E94C30B80E001C081E0EF
:1026C000DF91CF9108950F931F93CF93DF93C42F82
:1026D000D22FFC0182818823C9F040933C020E94E2
:1026E000601590933B0280933A0280E28C0F883011
:1026F00008F057C0C77081E001C0880FCA95EAF79B
:10270000DF91CF911F910F910C949A0380913C021D
:10271000481330C080913A0290913B020E94781594
:10272000883C910538F510E21D0FCD17B9F080E215
:102730008C0F883040F4C77081E001C0880FCA95C3
:10274000EAF70E94A103183028F581E09D2F9770C9
:1027500001C0880F9A95EAF70E949A03802F0E9481
:1027600091031830F0F4D77081E001C0880FDA953A
:10277000EAF70AC080E28C0F883098F4C77081E0D5
:1027800001C0880FCA95EAF7DF91CF911F910F9191
:102790000C94A103802FDF91CF911F910F910C9486
:1027A0009103DF91CF911F910F9108950F939C0199
:1027B000CB01243F4CE5340731F188F4293DFCE599
:1027C0003F07D9F02A3D4CE5340779F1283D3C45D7
:1027D000A9F506E221EE41EE68ED7CE52BC0263F2F
:1027E000FCE53F07E1F0A8F0273F3C4539F507E25B
:1027F00025EE46EE67EF7CE51DC007E225EE45EECF
:1028000069ED7CE517C006E221EE40EE64EF7CE561
:1028100011C007E225EE44EE65EF7CE50BC006E251
:1028200021EE42EE66EF7CE505C008E221E045EED0
:102830006AED7CE50E94631380E008C0FC018281A0
:10284000882319F010923C0201C081E00F91089595
:1028500090938B0180938A01089590934202809314
:1028600041020895E0914102F0914202309721F037
:102870000190F081E02D099480E00895E0914102FB
:10288000F0914202309721F00280F381E02D09940B
:10289000089520913F02309140022817390771F0C6
:1028A0009093400280933F02E0914102F0914202F6
:1028B000309721F00680F781E02D0994089520914A
:1028C0003D0230913E022817390771F090933E0285
:1028D00080933D02E0914102F0914202309721F055
:1028E0000084F185E02D09940895FC01329697E06B
:1028F00080E0915029F021912223D9F38F5FF9CF05
:102900000895662349F0FC013296089621916217DA
:1029100029F0E817F907D1F780E0089581E00895DC
:102920009C01FC0132969FEF80E04191461789F0AF
:102930009F3F19F4411101C0982F8F5F8630A9F78E
:102940009F3F39F0F901E90FF11D97FDFA95628378
:10295000089508959C012A5F3F4FFC014281461370
:1029600001C01282019682179307B9F708950C945B
:1029700090140C94AA14029626E0FC0111922A9558
:10298000E9F7089508950C94C21483E080934302FC
:102990000C94C314811102C081E001C082E08093D5
:1029A00043020C94C3140C94CA1481E08093430234
:1029B0000C94C3140C94D51408950C94DC140C944A
:1029C000DD140C94DC140C94DC140C94DC14CF9304
:1029D0000E94E3140E9449110E94E114C0E08C2F70
:1029E0000E945410672B682B692B29F4CF5FC530E8
:1029F000B1F780E001C081E0CF91089508951F9262
:102A00000F920FB60F9211248F939F93AF93BF93A2
:102A100080914402811113C080917C0290917D02CB
:102A2000A0917E02B0917F024196A11DB11D8093BD
:102A30007C0290937D02A0937E02B0937F02BF91AF
:102A4000AF919F918F910F900FBE0F901F9018958F
:102A500080918402843031F10E94850210924402F8
:102A600020E488E190E00FB6F894A8958093600088
:102A70000FBE2093600083B7817F846083BF83B7DC
:102A8000816083BF7894889583B78E7F83BF0FB6AC
:102A9000F894A895809160008861809360001092FE
:102AA00060000FBE08950E942E060C94890282E0F9
:102AB00084BD93E095BD9AEF97BD80936E00089515
:102AC0002FB7F89480917C0290917D02A0917E02B4
:102AD000B0917F022FBF08952FB7F89460917C02C8
:102AE00070917D0280917E0290917F022FBF0895A8
:102AF0009C014FB7F89480917C0290917D02A09147
:102B00007E02B0917F024FBF821B930B0895789491
:102B10001F920F920FB60F9211248F939F93AF9332
:102B2000BF9380917C0290917D02A0917E02B09132
:102B30007F020196A11DB11D80937C0290937D02BE
:102B4000A0937E02B0937F02BF91AF919F918F912E
:102B50000F900FBE0F901F90189581E08093E000BA
:102B600080E28093D8001092C9008FE19EE4019723
:102B7000F1F700C0000087E090EBDC0180938D024C
:102B800090938E02A0938F02B09390029CE088E114
:102B90000FB6F894A895809360000FBE90936000E4
:102BA000FFCF8091500208950895CF93DF9321E0E5
:102BB0002093E9002FEF3091E800215035FD06C049
:102BC00035ED3A95F1F700002111F5CF2091E8009D
:102BD00025FF14C0EC0140E050E068E070E00E9486
:102BE000E1178091E8008E778093E80088E0FE018D
:102BF000A8E4B2E001900D928A95E1F7DF91CF91C0
:102C00000895809345027093470260934602809135
:102C10008402843001F582E08093E9008FEF909187
:102C2000E800815095FD06C095ED9A95F1F70000FA
:102C30008111F5CF8091E80085FF0DC040E050E0A4
:102C400063E070E085E492E00E94E1178091E80083
:102C50008E778093E8000895BC0184E00C940116FF
:102C6000BC0183E00C9401160895809183028111C8
:102C700009C00E9472190E94CF198091E2008460FD
:102C80008093E20008951092830208950C94DA1460
:102C90006091800281E0611101C080E00C94C51454
:102CA0009091840281E0943009F080E0609180028C
:102CB0000C94CA1442E061EC81E00E94EB1842E2FD
:102CC00061EC82E00E94EB189091840281E09430E4
:102CD00009F080E0609180020C94D3148091860208
:102CE000833009F461C030F4813071F0823009F42E
:102CF0009AC008958A3009F486C08B3009F46CC0FC
:102D0000893009F0A8C020C080918502813A09F07D
:102D1000A2C08091E800877F8093E80080918902BB
:102D200090918A02892B21F468E088E492E003C044
:102D300060E080E090E070E00E942C188091E80054
:102D40008B778093E800089580918502813209F0A5
:102D500082C08091890290918A02029708F07BC01C
:102D60008091E800877F8093E8008091E80082FDF1
:102D700005C0809184028111F8CF6DC02091F300CD
:102D80008091F20090E0922B029731F48091F10053
:102D9000813011F0863021F48091F100809350024F
:102DA0008091E8008B7753C080918502813A09F0C9
:102DB00052C08091890290918A02892B09F04BC000
:102DC0008091E800877F8093E8008091E80080FF91
:102DD000FCCF8091100136C0809185028132D9F5F7
:102DE0008091890290918A02892BA9F58091E8004F
:102DF000877F8093E8000E9420198091870280934A
:102E000010010C942E0680918502813221F580916B
:102E1000E800877F8093E8000E9420198091880253
:102E200080935102089580918502813AA1F48091A6
:102E3000E800877F8093E8008091E80080FFFCCF66
:102E4000809151028093F1008091E8008E77809309
:102E5000E8000C942019089584B7877F84BF0FB6CB
:102E6000F894A8958091600088618093600010922A
:102E700060000FBE90E080E80FB6F8948093610088
:102E8000909361000FBE0C94D5140E9472190E9499
:102E9000CF19E2EEF0E080818460808378940C9416
:102EA000641C84E091E00C942D14809184028530A0
:102EB000A9F480918402853079F40E9428158091CC
:102EC00082028823B1F30E94E714882391F30E94C1
:102ED000CB170E942E06EDCF0C945315089508953C
:102EE0000C947217292F332723303105C9F060F471
:102EF0002130310581F02230310509F044C08BE3E7
:102F000090E026E632E043C021323105E1F0223282
:102F1000310549F138C082E190E021EA32E037C062
:102F200099278130910549F028F0029761F5ECE28C
:102F3000F2E005C0E2E6F2E002C0EAE4F2E08491E9
:102F400090E09F0124C06115710541F06130710569
:102F5000D1F489E090E021E932E019C089E090E005
:102F600028E732E014C06115710541F06130710548
:102F700051F482E390E023EB32E009C080E490E07A
:102F800025EE32E004C080E090E020E030E0FA017D
:102F900031832083089580E189BD82E189BD09B430
:102FA00000FEFDCF8091D8008F7D8093D800809166
:102FB000E00082608093E0008091E00081FDFCCF22
:102FC0000895CF92DF92EF92FF920F931F93CF93CA
:102FD000DF93EC018B017A010E943F19811133C00C
:102FE000E114F10439F0F70180819181081B190B7C
:102FF000C80FD91FC12CD12C0115110519F18091D1
:10300000E80085FD16C08091E8008E778093E80087
:10301000E114F10449F0F70180819181C80ED91EB5
:10302000D182C08285E00FC00E943F19882321F31E
:103030000AC089918093F10001501109FFEFCF1A66
:10304000DF0ADACF80E0DF91CF911F910F91FF90DF
:10305000EF90DF90CF90089520918B0230918C02F9
:103060002617370748F06115710539F42091E800FB
:103070002E772093E80001C0B901FC0120E0611522
:10308000710579F1809184028823F1F18530F1F1A5
:103090008091E80083FD3CC08091E80082FD2EC055
:1030A0008091E80080FFEBCF2091F3008091F20047
:1030B00090E0922B6115710551F08830910538F43C
:1030C00021912093F100615071090196F3CF21E025
:1030D000089709F020E08091E8008E778093E8005F
:1030E000CECF2111CFCF0AC080918402882361F016
:1030F000853061F08091E80083FD0AC08091E8008E
:1031000082FFF2CF80E0089582E0089583E0089581
:1031100081E0089520918B0230918C0226173707A9
:1031200048F06115710539F42091E8002E7720935D
:10313000E80001C0B901FC0120E06115710591F1C1
:1031400080918402882309F440C0853009F43FC08F
:103150008091E80083FD3DC08091E80082FD2FC092
:103160008091E80080FFE9CF2091F3008091F20088
:1031700090E0922B6115710559F08830910540F46B
:1031800024912093F1003196615071090196F2CF9C
:1031900021E0089709F020E08091E8008E77809385
:1031A000E800CBCF2111CCCF0AC0809184028823C4
:1031B00061F0853061F08091E80083FD0AC0809164
:1031C000E80082FFF2CF80E0089582E0089583E076
:1031D000089581E00895982F973068F59093E9005D
:1031E000981739F07091EC002091ED005091F000AB
:1031F00003C0242F762F50E021FD02C09F5FECCF4B
:103200003091EB003E7F3093EB003091ED003D7F3D
:103210003093ED003091EB0031603093EB00709310
:10322000EC002093ED005093F0002091EE0027FD7C
:10323000E5CF80E008958F708093E90081E00895E4
:103240008091850287FF11C08091E80082FD05C052
:10325000809184028111F8CF11C08091E8008B77B2
:103260000BC080918402882349F08091E80080FFA0
:10327000F8CF8091E8008E778093E8000895209140
:10328000E4003091E50095E64091EC00842F8170D8
:1032900040FF23C08091E80080FD1DC08091840222
:1032A000882399F0853099F08091EB0085FD11C05D
:1032B0004091E4005091E5002417350729F391501F
:1032C00011F09A01E1CF84E0089582E0089583E04F
:1032D000089581E0089580E008954091E80042FF5C
:1032E000DDCF08950E94E0190E94E819E0EEF0E0B9
:1032F000808181608083E8EDF0E080818F7780833A
:1033000019BCA7EDB0E08C918E7F8C9380818F7E6D
:1033100080831092830208950F931F93CF93DF93BE
:103320000E94E0190E94E819C8EDD0E088818F77EB
:10333000888388818068888388818F7D888319BC91
:1033400010928402109280021092820210928102E6
:1033500000EE10E0F80180818B7F8083888181609E
:10336000888342E060E080E00E94EB18E1EEF0E04C
:1033700080818E7F8083E2EEF0E0808181608083B7
:10338000808188608083F80180818E7F808388813E
:1033900080618883DF91CF911F910F910895E8EDAF
:1033A000F0E080818F7E8083E7EDF0E080818160B6
:1033B000808384E082BF81E0809383020C948C1927
:1033C000E8EDF0E080818E7F80831092E200089526
:1033D0001092DA001092E10008951F920F920FB63A
:1033E0000F9211242F933F934F935F936F937F938B
:1033F0008F939F93AF93BF93EF93FF938091E100DF
:1034000082FF0BC08091E20082FF07C08091E10043
:103410008B7F8093E1000E94631C8091DA0080FF23
:103420001FC08091D80080FF1BC08091DA008E7F82
:103430008093DA008091D90080FF0DC080E189BDC2
:1034400082E189BD09B400FEFDCF81E08093840252
:103450000E94351605C019BC109284020E944316C2
:103460008091E10080FF19C08091E20080FF15C0CB
:103470008091E2008E7F8093E2008091E200806183
:103480008093E2008091D80080628093D80019BCBC
:1034900085E0809384020E9448168091E10084FFB9
:1034A00030C08091E20084FF2CC080E189BD82E1C0
:1034B00089BD09B400FEFDCF8091D8008F7D809337
:1034C000D8008091E1008F7E8093E1008091E2003E
:1034D0008F7E8093E2008091E20081608093E20021
:1034E00080918002882311F084E007C08091E3007E
:1034F00087FD02C081E001C083E0809384020E94C6
:1035000050168091E10083FF29C08091E20083FF83
:1035100025C08091E100877F8093E10082E0809365
:103520008402109280028091E1008E7F8093E100FE
:103530008091E2008E7F8093E2008091E2008061C2
:103540008093E20042E060E080E00E94EB1880910E
:10355000F00088608093F0000E944616FF91EF9182
:10356000BF91AF919F918F917F916F915F914F919B
:103570003F912F910F900FBE0F901F9018951F92A3
:103580000F920FB60F9211242F933F934F935F9397
:103590006F937F938F939F93AF93BF93CF93DF935B
:1035A000EF93FF93C091E900CF708091EC00D82F8A
:1035B000D17080FDD0E81092E9008091F000877F03
:1035C0008093F00078940E94031B1092E900809190
:1035D000F00088608093F000CD2BCF70C093E9009D
:1035E000FF91EF91DF91CF91BF91AF919F918F911B
:1035F0007F916F915F914F913F912F910F900FBEEF
:103600000F901F9018951F93CF93DF93CDB7DEB720
:10361000AA970FB6F894DEBF0FBECDBFE5E8F2E083
:103620008091F100819322E0ED38F207C9F70E9402
:103630006E168091E80083FF2EC1809185029091E3
:103640008602492F50E04A30510508F024C1FA01A2
:10365000EE59FF4F0C947F1C803821F0823809F01E
:103660001AC108C08091810290918202992389F049
:1036700082600FC0809189028F70873008F00BC183
:103680008093E9008091EB0085FB882780F91092F8
:10369000E9009091E800977F9093E8008093F10013
:1036A0001092F100D1C0282F2D7F09F0F4C088239B
:1036B00019F0823061F0EFC080918702813009F00B
:1036C000EAC0933009F080E0809382022EC080919E
:1036D000870281112AC0809189028F702FEF280FF5
:1036E000263008F0D8C08093E9002091EB0020FF3D
:1036F0001CC0933021F48091EB00806214C0909143
:10370000EB0090619093EB0021E030E0A90102C052
:10371000440F551F8A95E2F74093EA001092EA00A1
:103720008091EB0088608093EB001092E90080911B
:10373000E800877F8093E8000E942019ACC08111C7
:10374000AAC0109187021F778091E3008078812BB7
:103750008093E3008091E800877F8093E8000E94D7
:1037600020198091E80080FFFCCF8091E300806801
:103770008093E300111102C082E001C083E08093D6
:10378000840289C08058823008F085C08091870209
:10379000909188028C3D53E0950779F583E08A8308
:1037A0008AE289834FB7F894DE01139620E03EE069
:1037B00051E2E32FF0E050935700E49120FF03C063
:1037C000E295EF703F5FEF708E2F90E0EA3010F0DF
:1037D000C79601C0C0968D939D932F5F243149F702
:1037E0004FBF8091E800877F8093E8006AE270E035
:1037F000CE0101960E942C1816C06091890270912A
:103800008A02AE014F5F5F4F0E947017BC01892B87
:1038100009F441C09091E800977F9093E800898176
:103820009A810E948A188091E8008B778093E80043
:1038300032C0803881F58091E800877F8093E8006E
:10384000809180028093F1008091E8008E7772CFA2
:10385000811121C080918702909188029927029757
:10386000D4F48091E800877F8093E80080918702FC
:10387000809380020E94201980918002811106C0ED
:103880008091E30087FD02C081E001C084E0809365
:1038900084020E945A168091E80083FF0AC080913A
:1038A000E800877F8093E8008091EB00806280933E
:1038B000EB00AA960FB6F894DEBF0FBECDBFDF9126
:1038C000CF911F9108950895CF938091840288230A
:1038D000A1F0C091E900CF709091EC00892F817028
:1038E00090FD80E8C82B1092E9008091E80083FDEC
:1038F0000E94031BCF70C093E900CF910895EE0F93
:10390000FF1F0590F491E02D0994FB01DC0104C038
:103910008D910190801921F441505040C8F7881BC7
:10392000990B0895F999FECF92BD81BDF89A992718
:1039300080B50895A8E1B0E042E050E00C94C61CC8
:10394000262FF999FECF92BD81BDF89A019700B458
:10395000021639F01FBA20BD0FB6F894FA9AF99AF8
:103960000FBE08950396272F0E94A11C0E94A01C41
:10397000252F0E94A11C242F0C94A11C0196272FF7
:103980000E94A11C0C94A01CDC01CB01FC01F99944
:10399000FECF06C0F2BDE1BDF89A319600B40D929B
:0C39A00041505040B8F70895F894FFCF54
:1039AC00C8000F02D115D515341630162C16D415A7
:1039BC0001E200E900EA00B500B600B700CD0083D3
:1039CC0001CC008A019201940121022302240225D8
:1039DC0002260227022A02B300B4006F0070008195
:1039EC008283E200E900EA00B500B600B700CD0022
:1039FC008301CC008A01920194012102230224024A
:103A0C002502260227022A02B300B4006F007000C0
:103A1C0081828394969734353666F5F4F1F0313221
:0A3A2C0033929395919030F6F70065
:00000001FF
